:040000006F00C0408D
:100004000000000000000000480200004A02000056
:10001400000000000A0400000000000000000000CE
:100024000A0400000A0400000000000000000000B0
:100034000A040000000000000A04000000000000A0
:100044000A0400000A0400000A0400000A04000074
:100054000A0400000A0400000A0400000A04000064
:100064000A0400000A0400000A0400000A04000054
:100074000A0400000A0400000A0400000A04000044
:100084000A0400000A0400000A0400000A04000034
:100094000A0400000A0400000A0400000A04000024
:1000A4000A0400000A0400000A0400000A04000014
:1000B4000A0400000A0400000A0400000A04000004
:1000C4000A0400000A0400000A0400000A040000F4
:1000D4000A0400000A0400000A0400000A040000E4
:1000E4000A0400000A0400000A0400000A040000D4
:1000F4000A0400000A0400000A0400000A040000C4
:100104000A0400000A040000000000000A040000C1
:100114000A040000000000000000000000000000CD
:1001240000000000000000000000000000000000CB
:0C013400000000000000000000000000BF
:10014000397101436EC619A0397141536AC866CA34
:1001500062CC5ECE19A0397101535AD056D252D416
:100160004ED64AD826DA22DC06DE3301614082828E
:1001700041114AC026C222C406C68282B24D410144
:10018000024D924C224CB24B4101024B924A224A00
:10019000B2494101024992442244B2404101828065
:1001A0003D432A876373C3029377F700BDEFADE544
:1001B000937606FF3D8ABA960CC34CC30CC74CC756
:1001C0004107E36BD7FE11E28280B306C3408A0683
:1001D0009702000096966780A6002307B700A30643
:1001E000B7002306B700A305B7002305B700A30493
:1001F000B7002304B700A303B7002303B700A3028B
:10020000B7002302B700A301B7002301B700A30082
:10021000B7002300B700828093F5F50F9396850011
:10022000D58D93960501D58D61B7939627009702DA
:10023000000096968682E78086FA9680C1171D8F09
:100240003E96E374C3F8A5B701A0B707EFBE37E742
:1002500000E0938707083CC701A0EFF27FF1054556
:10026000DD231122EF00E07B716513050520EF000F
:10027000B000B707002083A5070837250000130545
:1002800005CEEF00900A3124AA853725000013051A
:1002900005CFEF009009372400001305803EEF00E2
:1002A000407A130504D0EF009019C5BFEFF25FEC60
:1002B000371402401C403707FF0893E717001CC0A3
:1002C0005C40F98F5CC01C403707F7FE6D17F98F53
:1002D0001CC01C403707FCFF7D17F98F1CC05C4019
:1002E000370701FF7D17F98F5CC0B7079F001CC45B
:1002F000512EB7270240094798C33747024083274A
:10030000078093E707012320F7805C403707C1FF90
:100310007D175CC05C405CC05C4093E707405CC0FC
:100320005C40F98F5CC05C4037072800D98F5CC007
:100330001C4037070001D98F1CC0B71702409843F3
:1003400093166700E3DD06FED843B7160240719BA3
:10035000D8C3D84313672700D8C32147DC42B18BE9
:10036000E39EE7FE05BDB7160240DC4237070020DA
:100370001146B18B13070708638FC70221466381BB
:10038000C70495EB9C42918B9DC7B7470F0093879D
:1003900007241CC3B7170240DC43918393F6F70090
:1003A000B707002093870700B69794231C43B3D761
:1003B000D7001CC38280B7177A0093870720D1BF6C
:1003C000DC42D4424166C983BD8BF18E8907454624
:1003D0006393C700C94781EEB746024083A60680F3
:1003E000C18A89CEB7167A009386062021A8B7164F
:1003F0000240D4421396E600E35606FEB7163D00CF
:1004000093860690B387D70269B701A097010020B1
:1004100093814147175100201301C1BE17250000E9
:100420001305C599970500209385C5BD1386818165
:1004300063FAC5008322050023A05500110591052C
:10044000E3EAC5FE13858181938501846377B50056
:10045000232005001105E36DB5FEFD42739002BC3B
:100460008D4273904280930280087390023097020D
:100470000000938262B993E2320073905230EFF041
:10048000FFE297020000938282DD739012347300C2
:10049000203003A5C18182809C4513F7070113F822
:1004A000F70001C7D8413368E8008E2113F7F50F34
:1004B00039C318418146854E3D4F930F8002930208
:1004C0008004214E3396DE00B3F8C5006311160395
:1004D0009398260033131F011343F3FF3377E30090
:1004E000B318180133E7E800639FF70550C9850684
:1004F000E39AC6FD18C11307F00F6375B7045441A2
:100500002146854E3D4F930F800293028004414E59
:10051000B398CE0033F715016392E8021317260053
:1005200001173313EF001343F3FFB376D3003317F0
:10053000E800D98E639DF701232A15010506E3190A
:10054000C6FD54C18280E39457FA10C94DB7E397B2
:1005500057FE23281501DDB7370700C0B377E50044
:100560006395E708370701405C439356B501584F40
:100570009D8A9DE6F99BB70600FFFD16758F89C918
:1005800093160501C182D58FB706FF01758D498F7E
:10059000B7060007D58FB7060140DCC2D8CE8280EF
:1005A00005466396C600F59BB70680FFF9B7094676
:1005B0006396C600ED9BB706E8FFC1B70D4663968C
:1005C000C600DD9BB706FCFF4DBF11466397C60012
:1005D00093F7F7F3B706C0FF4DB71546E391C6FA98
:1005E00093F7F7CFB706E0FF49BF370700406391A5
:1005F000E702B7070140D84F4205B367A70089E576
:100600001345F5FFB377E500370701405CCF8280E3
:10061000A9E337080140B707300003264800131745
:100620000501B376F50041836396F602B70600F93B
:10063000FD16B377D60003264800F18E2322D8009A
:1006400091C5558112053315A700C98F37070140A1
:100650005CC382809317B50063D0070293570501EE
:1006600093F6F7008D47B397D70093C7F7FFF18F45
:10067000B7060007D58FE9B7935755019207B3170F
:10068000F700E5B7EFF2DFAE37F4FF1F0327447240
:100690003706003E4111931797019346F7FFF18FFC
:1006A000060737063E00718FD98F37060001139772
:1006B0009600718FD98FBD824167F98E02C202C444
:1006C00002C6D58F23A0F182035784728545239CEF
:1006D000E180032704721305D00323A2E1820327DC
:1006E000447023AEE180035704732394E182152CF8
:1006F0008327447037073A101307077093F7F7F012
:100700006383E710636AF700370732101307077037
:10071000638FE7064101BDBC37073B101307077025
:10072000638BE70837073D1013070770E394E7FE74
:1007300085452165153537140140E1779304800420
:100740004C00130504807C8226C6B93385679387E5
:1007500087334C00130504C07C8226C6353B914785
:100760007C824C0093078002130504C03EC62D33E3
:10077000F9774C00371501407C8226C6313B8D4706
:100780007C8226C64C0013050440393361B7E177FB
:100790003715014093C707C0130480044C001305AC
:1007A00005C07C8222C6CD3989677C8222C64C0076
:1007B00037150140D9BF85452165793B3714014084
:1007C000E177930480044C00130504807C8226C6E4
:1007D000E131930700214C00130504C07C8226C63A
:1007E000653991477C824C0093078002130504C051
:1007F0003EC65D31F9774C00371501407C8226C634
:1008000061398947B5BFB7140140E1779387077015
:10081000130480044C00138504807C8222C6AD3909
:10082000930790E34C00138504C07C8222C6AD314F
:1008300091477C824C0093078002138504C03EC61A
:10084000A139F9779DB723A6A1828280371702408C
:100850005C439146B18B638CD706A146638ED70665
:10086000BDE71C43918BA5C7B7470F0093870724AB
:100870001CC1371602405C423707002013070701EE
:100880009183BD8BBA9794231C41B3D7D7005CC129
:100890005442A1829D8ABA969422B3D6D70014C539
:1008A0005442AD829D8A36971423B3D6D70054C5DF
:1008B0005842634C07005C42B98313F737009387B3
:1008C0004180BA979C23B3D7F6021CC98280B71720
:1008D0007A009387072069BF5C435843C166C98388
:1008E000BD8B758F8907C5466393D700C94701EF54
:1008F0003747024003270780418B09CF37177A001B
:100900001307072021A83717024058439316E70022
:10091000E3D606FE37173D0013070790B387E702BB
:1009200081BF99C5371702401C4F5D8D08CF82806B
:10093000B7170240984F1345F5FF798D88CF828015
:10094000EFF21F831629F577FD17F58FF621DA25CB
:100950007971D58F1EA95625FD779387379FF58F1F
:10096000D6212A842EC6D58F9625D58FB625D58F2C
:100970005EA55E29C207C18393F7F7CFD98F5EA921
:100980006808E935B747014093870780B245631A85
:10099000F404A25756246547B387E702C206C1860E
:1009A000984163D20604060752244206B3D7E702F1
:1009B000130740064186B3D6E702B3F7E702920673
:1009C000635506028E0793872703B3D7E70213F711
:1009D0007700B367D700C207C1831EA445616FF0DB
:1009E0006FFB925745BF0A07C1B79207938727034A
:1009F000B3D7E702BD8BD58FF9BF91C55E250967D7
:100A0000D98F5EA582805A25F977FD17F98FD5BF5A
:100A100093F5F51F4EA182800A216D8D3335A0001C
:100A20008280B707002083A707080967130707F428
:100A3000B3D7E702C207C1832399F1822398F182D9
:100A40008280B7F700E0D8438146799BD8C303D7AB
:100A500001833306A70290CBD4CB984313670701D9
:100A600098C398431367170298C3D843058B75DF63
:100A70009843799B98C38280EFF28FEF2A841165A7
:100A8000011185451105713D930700207C823715C2
:100A900001408D473EC44C00E147130505803EC62A
:100AA000E53A22C837440140B70708000C0813058F
:100AB00004803ECC02CA231E01005935854513052A
:100AC0000480253F05616FF0EFECEFF2CFE8B7440B
:100AD0000140AE8932890144938404806345240136
:100AE0004A856FF08FEA930500042685353765DD6A
:100AF000B38789008385070026850504C205C18167
:100B0000013FE9BF138781801C43938601843E9592
:100B1000636BD500B75600209386068063E5A60078
:100B200008C33E858280FD57EDBF39713EDA2ED273
:100B300032D436D63AD842DC46DE9387C18022CC06
:100B4000804326CA06CEAA8409C41C4C99E3228598
:100B5000ED290C4454102686228536C6EF0070120B
:100B6000F2406244D24421618280011126CA4AC8FF
:100B700006CE22CC4EC652C4AA842E8901C51C4D75
:100B800091E3E1219C4C804499E326857D299717C8
:100B900000009387E71A631BF402C0405E24A18B18
:100BA000B1C71C48A1C7FD59294A1C448345090007
:100BB000FD17B1E91CC463DD07062286A945268519
:100BC0006120FD576308F502294535A097170000FD
:100BD000938707196314F4008044C9B7971700007E
:100BE00093870714E31CF4FAC0444DBFA285268501
:100BF000112A55D97D55F2406244D2444249B24946
:100C0000224A056182801CC4050963D70700184C7D
:100C100063CAE700638845011C401387170018C0AA
:100C20008CA361B7228626850520E31035F9D9B754
:100C30001C401387170018C0294798A371B79387E2
:100C4000C180AA85884315B7011122CC26CA4AC89B
:100C500006CE4EC6AA842E89328401C51C4D91E36E
:100C6000ED26971700009387A70D6317F406C04081
:100C70001C4C1CC45E24A18BC1C31C48B5CF1C48AE
:100C800008409379F90F1379F90F1D8D5C4863467D
:100C9000F500A2852685692C25E51C440505FD1770
:100CA0001CC41C401387170018C0238037015C4800
:100CB0006388A7005E24858B81CBA9476316F90062
:100CC000A2852685B5240DEDF24062444A85D244C2
:100CD0004249B2490561828097170000938747080F
:100CE0006314F400804469B79717000093874703A3
:100CF000E310F4F8C044ADBFA2852685212041D180
:100D00007D59D9B741119387C18026C2844322C43B
:100D10004AC006C62A892E8489C49C4C99E326853C
:100D20002D26971700009387A701631BF402C0408C
:100D30000317C40093170701C18393F68700ADEA38
:100D400093F6070195EEA5472320F90013670704E2
:100D50005AA47D55B2402244924402494101828006
:100D6000971700009387C7FF6314F4008044C9B746
:100D7000971700009387C7FAE31CF4FAC0444DBFED
:100D8000918B9DC34C5889C9930744046384F50033
:100D90004A853123232A04025E242322040093F788
:100DA000B7FD5EA41C481CC05E2493E787005EA4C8
:100DB0001C4899EB5E241307002093F707286385EE
:100DC000E700A2854A85A1215E2413F717001DC301
:100DD0005C4823240400B307F0401CCC1C480145A8
:100DE000B5FB8317C40013F707082DD793E7070453
:100DF0005EA485B7898B014791E3584818C4F9BFB1
:100E0000DE25011122CC26CA06CE4AC84EC613F7EB
:100E10008700AA842E8479EBD841634DE000B84165
:100E2000634AE0000145F2406244D2444249B2497B
:100E30000561828058547DD703A904009396370139
:100E400023A0040063DB060670485E24918B99C7DB
:100E50005C401D8E5C5899C33C401D8E5C540C5008
:100E6000814626858297FD575A24631DF5009440DC
:100E7000F54763E8D706B70740208507B3D7D70003
:100E8000858BA5C31C48232204001CC0931737017F
:100E900063D80700FD576314F5009C4091E368C8D0
:100EA0004C5823A02401BDDD930744046384F5005E
:100EB0002685F526232A0402B5B70C50014685463F
:100EC00026850297FD572A86E311F5F89C40B5DF89
:100ED00075476385E70059476393E70423A024011E
:100EE00091B7136707045AA47D5535BF83A905013F
:100EF000E38A09F203A905008D8B23A0350133098C
:100F00003941014791E3D84918C4E35D20F11C54ED
:100F10000C50CA864E86268582976347A0005E24C1
:100F200093E707045EA4C9B7AA993309A940F1BFA2
:100F30009C49B9CF011122CC06CE2A8411C51C4D83
:100F400081E72EC61922B24597170000938747DF25
:100F5000639BF5004C408397C50095C7228562448A
:100F6000F240056171BD97170000938767DF6394B6
:100F7000F5000C44CDB797170000938767DAE39C20
:100F8000F5FC4C44C9BFF2406244014505618280D2
:100F900001458280411122C406C62A844EA572A54D
:100FA0002320050023220500232405002322050613
:100FB00023280500232A0500232C0500214681450E
:100FC0001305C505EFF0CF9D97170000938747B134
:100FD0005CD097170000938767B31CD49717000065
:100FE000938747B75CD4971700009387A7B900D0C1
:100FF0001CD8B240224441018280970500009385AD
:1010000065F3A9A2411126C2130680069384F5FF59
:10101000B384C4024AC02E8922C406C693854407FD
:101020001D262A8401CD2320050023222501310518
:1010300008C4138684068145EFF08F962285B2405E
:10104000224492440249410182801C4DADE341118A
:1010500006C622C497070000938767FA1CD59387BA
:1010600001819C4323240504232605042328050429
:101070006314F50085471CCD2A841D2848C02285AD
:10108000052808C422852D2048C4484001469145C2
:10109000113708440546A545F53D48440946C9456C
:1010A000D53D85471CCCB2402244410182808280DC
:1010B00041119387018126C284434AC006C69C4CD5
:1010C00022C42A8999E3268549379384840480447D
:1010D000DC40FD1763D607009C40B9CF8440C5BFF4
:1010E0000317C40039E7C1778507232204062320AC
:1010F000040023220400232404005CC423280400E9
:10110000232A0400232C0400214681451305C4052D
:10111000EFF00F89232A0402232C04022324040461
:10112000232604042285B24022449244024941010C
:1011300082801304840671BF91454A85E13588C0D9
:1011400051FDB1472320F9000144E9BF797122D450
:101150004AD052CC56CA5AC85EC606D626D24ECE01
:101160002A8AAE8A130485040149054BFD5B09EC0C
:10117000B25022544A8592540259F249624AD24AE4
:10118000424BB24B45618280044483294400FD19DF
:1011900063D409000040E1BFDE24637BFB0083973A
:1011A000E40063877701A6855285829A3369A90096
:1011B00093848406E9BF1971A6DAAE848395E500AD
:1011C000A2DC86DE328463DB0500DE2423A0060079
:1011D00093F7070885E7930700401DA0300836C63F
:1011E000EF00D01FB246E34205FE7247BD67F98F9C
:1011F0007977BA9793B717009CC2F1BF93070004A1
:101200001CC0F6506654D654014509618280DE2523
:10121000011122CC06CE26CA4AC8898B2E8489CFDA
:10122000930774041CC01CC885475CC8F240624424
:10123000D24442490561828074003000AA84A53FEF
:10124000A2452A892685012219E98317C40013F7CC
:10125000072069FFF19B93E727005EA4D1B79707AA
:1012600000009387C7D99CD45E2408C008C893E7C0
:1012700007085EA4A2475CC8B24781CF8315E4008B
:101280002685EF00501811C55E24F19B93E71700E7
:101290005EA45E243369F9002316240141BFDDC139
:1012A00083A7C5FF411122C406C626C21384C5FF09
:1012B00063D307003E94AA84EF00B01B9387418359
:1012C0009C4381EF2322040023AA81822244B2405E
:1012D0002685924441016F00F019637EF4001440AA
:1012E0003307D4006396E7009843DC43369718C071
:1012F0005CC0D9BFBA87D84319C3E37DE4FE9443E9
:101300003386D700631F86001040B29694C333869D
:10131000D700E31DC7FA10435843B29694C3D8C30D
:1013200075B76375C400B1479CC04DB71040B30694
:10133000C4006316D70014435843B29614C058C073
:10134000C0C369B78280011126CA93843500F19821
:1013500006CE22CC4AC84EC6A104B14763F3F404BA
:10136000B14463E2B4042A89EF00B010938741834B
:1013700098433A8439E0938781839C4391E7814580
:101380004A85052F23ACA182A6854A851D27FD59D4
:1013900063193507B1472320F9004A85EF00900D06
:1013A00029A0E3D004FCB1471CC10145F2406244CE
:1013B000D2444249B249056182801C40858F63CF87
:1013C0000702AD4663F6F6001CC03E9404C031A08F
:1013D0005C406313870223AAF1824A85EF009009DB
:1013E0001305B4009307440061993307F5405DDFAE
:1013F0003A94898F1CC05DBF5CC3C5B7228740404B
:1014000095BF130435007198E30285FCB305A44031
:101410004A854525E31C35FBB5BF1C46FD171CC698
:1014200063DA0700184E63C5E700A9476394F50027
:101430006FF09F811C422E851387170018C28CA362
:101440008280011122CC26CA4AC84EC652C406CE9A
:101450002A89AE893284B304D6007D5A631494007D
:10146000014501A80C204E864A85453F0504E31737
:1014700045FFF2406244D2444249B249224A0561E2
:101480008280357122CD26CB4AC94EC706CF52C5C0
:1014900056C35AC1DEDEE2DCE6DAAA89AE843289BE
:1014A000368401C51C4D91E34D3697170000938794
:1014B00027896397F40C83A44900DE24A18BFDC324
:1014C0009C48EDC393070002A304F10293070003B5
:1014D00002D22305F10222C6930B5002971A000094
:1014E000938A0A8A054C294B4A841C2099C3639E1F
:1014F000770DB30C2441638D0C00E6864A86A685E1
:101500004E858137FD57630FF51C9256E69636D20D
:101510001C206389071CFD571309140002C802CE62
:101520003ECA02CCA309010482D4834509001546B2
:101530005685252713041900C24751E913F70701FF
:1015400009C713070002A309E10413F7870009C7BD
:101550001307B002A309E104834609001307A002A0
:10156000638FE606F2474A84814625461820930594
:101570001400130707FD6377E60AB5CA3ECE85A8B7
:10158000970700009387C77D6395F40083A48900C3
:101590002DB7970700009387A778E390F4F283A410
:1015A000C90021BFA6854E85EFF0CFF501DD7D5541
:1015B000FA406A44DA444A49BA492A4A9A4A0A4BE2
:1015C000F65B665CD65C0D618280050439BF33052D
:1015D00055413315AC00C98F3EC82289B9B732478F
:1015E00093064700184336C6634707023ACE1820D1
:1015F0009307E002631DF70418309307A002631BF2
:10160000F702B2470904138747009C433AC663C1F7
:1016100007023ECA2DA83307E04093E727003ACEE1
:101620003EC8F1B7B387670385462E84BA973DBF9E
:10163000FD57C5B7050402CA8146814725461820D3
:1016400093051400130707FD6374E606F9F20C20F6
:101650000D461705000013052573012511CD9707C9
:101660000000938767721D8D93070004B397A7004E
:10167000424505045D8D2AC80C2019461705000057
:101680001305C570130914002304B102F92335C1F1
:1016900097F7FFFF9387079795E74247B24713777E
:1016A000071009CF91073EC69257D2973ED22DBD63
:1016B000B387670385462E84BA9751B79D07E19B90
:1016C000A107D5B77800970600009386C6D726866F
:1016D0000C084E8597000000E7000000FD572A8A9D
:1016E000E314F5FCDE2493F70704E39207EC1255AC
:1016F000C1B57800970600009386E6D426860C08CC
:101700004E85012AE1BF797156CA9C49BA8A98452B
:1017100022D426D24ECE52CC06D64AD05AC85EC665
:10172000AA892E84B284368A63D3E700BA879CC024
:101730000347340419C385079CC01C4093F7070274
:1017400081C79C4089079CC0032904001379690064
:10175000631A0900130B9401FD5B5C449840998F58
:10176000634CF9041C408346340493F70702B336F4
:10177000D000A5EB13063404D2854E85829AFD571E
:101780006303F5041C4011469840998B54448144EE
:101790006397C700B384E64063D3040081441C44CC
:1017A00018486354F700998FBE94014969047D5B22
:1017B00063982405014509A885465A86D2854E8539
:1017C000829A631E75017D55B2502254925402597B
:1017D000F249624AD24A424BB24B456182800509C6
:1017E000ADBF3307D40013060003A301C7040347AA
:1017F000540493871600A2978906A381E7049DBF2E
:1018000085462286D2854E85829AE30E65FB0509C0
:1018100045B7797122D426D24AD04ECE06D652CCC4
:1018200056CA5AC8B689942D930790063289AA845D
:101830002E8413863504638DF60263E2D706930780
:1018400080056385F61863EDD700638D0620930746
:101850003004638EF60A930A24042301D404C9A039
:10186000930730066385F60A93074006E395F6FE74
:101870001C40084393F6070893054500C5C61C4164
:101880000CC363D807001307D002B307F040A301CD
:10189000E404970600009386E64F294765A893075E
:1018A00000076381F61663E5D7029307E0066388B5
:1018B000F6189307F006E390F6FA0C401C4313F871
:1018C0000508138547006307080608C39C4385A8DD
:1018D00093075007E383F6FE930780076388F612A9
:1018E00093073007E399F6F61C43D0418145938670
:1018F000470014C383AA07005685852601C5330512
:10190000554148C05C401CC8A301040461A81C43A5
:10191000930A2404938647009C4314C32301F404D0
:101920008547D5B793F607041C410CC3B9DAC20743
:10193000C18781BF93F5050408C3C9D99E23130746
:10194000F0066386E60E970600009386A6442947B4
:10195000A30104044C400CC463C5050008406D9904
:1019600008C099E3B28A89CDB28AB3F5E702FD1ABD
:10197000B6958C212380BA00B3D5E70263FFE70A4E
:10198000A147631EF7001C40858B91CB58401C4833
:1019900063C7E70093070003A38FFAFEFD1A33061F
:1019A000564110C84E87CA867000A2852685A13B85
:1019B0007D5A631D450B7D55B250225492540259F5
:1019C000F249624AD24A424B45618280A382D504E1
:1019D000970600009386063C0C40084313F8050860
:1019E0001C411105630D080208C313F7150001C758
:1019F00093E505020CC04147A1FF0C4093F5F5FDAE
:101A00000CC0B9B79C4193E707029CC193078007BC
:101A1000A302F404970600009386063975BF13F8F5
:101A2000050408C3E30308FCC207C1837DBF970612
:101A3000000093862636214721BFAE873DB79441EB
:101A40001C43CC4913F806081385470063060800B9
:101A500008C39C438CC339A008C393F606049C4377
:101A6000F5DA8EA323280400B28A2DBF14485686C7
:101A7000CA8526858299E30045F51C40898B8DE750
:101A8000B2474844E35AF5F23E853DB7854656864F
:101A9000CA8526858299E30065F3050A5C443247CE
:101AA000998FE345FAFEE9BF014A930A94017D5BF1
:101AB000F5B7411122C42A842E8523AE018206C6C1
:101AC000EFF04F84FD576317F5009387C1839C4364
:101AD00091C31CC0B240224441018280411122C402
:101AE0002E848395E50006C67922634905007C486B
:101AF000AA977CC8B2402244410182805E247D774F
:101B00007D17F98F5EA4FDB7DE25011122CC26CA10
:101B10004AC84EC606CE93F70710AA842E8432898F
:101B2000B68991C78395E5008946014609225E245E
:101B30007D777D17F98F5EA48315E4006244F2403F
:101B4000CE864A86B24942492685D244056125A8F7
:101B5000411122C42E848395E50006C6C928FD578D
:101B60005A24631AF500FD77FD17F98F5EA4B24081
:101B70002244410182808567D98F5EA468C8C5BFB1
:101B80008395E50005A8411122C42A842E85B285DB
:101B9000368623AE018206C6EFE03FF3FD5763179A
:101BA000F5009387C1839C4391C31CC0B24022447B
:101BB00041018280411122C42A842E8523AE0182F4
:101BC00006C6C520FD576317F5009387C1839C4364
:101BD00091C31CC0B240224441018280411122C401
:101BE0002A842E85B28523AE018206C6C920FD5700
:101BF0006317F5009387C1839C4391C31CC0B24017
:101C0000224441018280411122C42A842E8523AEC0
:101C1000018206C65D20FD576317F5009387C183D7
:101C20009C4391C31CC0B2402244410182804111B7
:101C300022C42A842E85B285368623AE018206C64A
:101C40005920FD576317F5009387C1839C4391C3C7
:101C50001CC0B24022444101828093F5F50F2A96C0
:101C60006314C500014582801C21E38EB7FE050583
:101C7000C5BF82808280411122C42A842E85B2850C
:101C8000368623AE018206C6A920FD576317F500EC
:101C90009387C1839C4391C31CC0B240224441013D
:101CA00082809307800523AEF1827D558280930761
:101CB000800523AEF1827D5582809307800523AE97
:101CC000F182014582809307800523AEF1827D5524
:101CD00082809307800523AEF1827D5582800000CB
:101CE00053797374656D436C6B3A25640D0A00007B
:101CF0004368697049443A253038780D0A0000007D
:101D000054686973206973207072696E7466206507
:101D100078616D706C652063630D00000000000049
:101D200000000000000000000000000000000000B3
:101D300000000000000000000000000000000000A3
:101D40000000000000000000000000000000000093
:101D50000000000000000000000000000000000083
:101D60000000000000000000000000000000000073
:101D7000000000000000000000000000232D302BB8
:101D800020000000686C4C0065666745464700000F
:101D900030313233343536373839414243444546A1
:101DA0000000000030313233343536373839616263
:081DB000636465660000000099
:101DB80000000000000000000102030406070809F3
:101DC80000000000010203040102030406070809D9
:101DD800000000003C1D00005C1D00001C1D0000F0
:101DE80000000000000000000000000000000000EB
:101DF80000000000000000000000000000000000DB
:101E080000000000000000000000000000000000CA
:101E180000000000000000000000000000000000BA
:101E280000000000000000000000000000000000AA
:101E380000D8B80502040608C000002020000020D1
:081E4800200000200000000052
:00000001FF
